:020000040000FA
:06000000FE300D303A282D
:08000800A000030EA100831209
:100010008B10851E4317851AC317210E8300A00E6F
:04002000200E0900A5
:0C007400203084008001840A80300402E7
:10008000031C3C280130E500E300D300E4004C10E1
:1000900083162E30850520308605003087058312B3
:1000A000850186018701103083168E00831270301F
:1000B00083168F008312003003179900031300305A
:1000C00003179A0003130030970000309F000030A0
:1000D00083169F008312003003179E000313003025
:1000E00003179F000313C030831681008312313041
:1000F000900000309200003083169400831200308C
:100100009400A630831698008312003083169B005B
:100110008312903098003330831699008312003098
:1001200083168C008312003083168D0083125030AA
:100130008B008B13063003178D0083168C130C1461
:1001400083120C080313F200F20381018E018F0168
:100150000B118B100B108C128C018D018B17C4208E
:1001600014232D233D215818C620581CE920512264
:100170008F080319AF288F0195226F22FB0BAF2840
:10018000FC0A7C195814AF2864000800D818062906
:10019000700AD100D20112215208D0004523D400A8
:1001A000591854175108D0004523D500D9185517B0
:1001B000710AD100D20112215208D0004523D60085
:1001C000591956175108D0004523D700D919571788
:1001D0000800720AD100D20112215208D000452332
:1001E000D4005108D0004523D5000930D100D201F8
:1001F00012215208D0004523D6005108D0004523D3
:10020000D70054175517561757170800A730D400B2
:100210004908D0004523D500D601D7015613D91976
:10022000571708000A305102031C0800D100D20AF7
:100230001229531C22294213C2138518421785190B
:10024000C2170800D31C2B294211C2118518421570
:100250008519C2150800531D3429C2104310851892
:10026000C214851943140800D31D08004212C2129B
:10027000851842168519C21608005910D910C418DD
:100280005914C41CD914461C472940145529401C34
:100290005429441344134517661467170130671F28
:1002A000E400DE226716E7164010441B5A15441F6F
:1002B0005911441F5A114C1CDA154C1C632958194A
:1002C000D915581DD911441B5A15441F5911441FE3
:1002D0005A11431CC310431C7129C3187129C3143C
:1002E000EA21421D4111421D8329411983294115EB
:1002F0000130C4064513C510451466146717013054
:10030000671FE400DE22C21DC111C21D9629C1195A
:100310009629C1150830C7064810C8104811C815DD
:10032000E61467170230671FE400DE22421E411206
:10033000421EA929411AA92941160130C7064814AD
:10034000C8104811C811661567170230671FE4000E
:10035000DE22C21EC112C21EBC29C11ABC29C1168E
:100360000230C7064810C8144811C811661567172F
:100370000230671FE400DE22FD0BC0295A08D906AF
:100380004A08CD054B08CE054E084B06FE004D0829
:100390004A06FF0000307E1B0830FE1A07307E1A26
:1003A0000630FE1905307E190430FE1803307E1821
:1003B00002307F180130C900C908D810031DD814B5
:1003C00058114A080139031D58154B087F39031D80
:1003D00058150800D8182D2A441BF32970087102FB
:1003E00003190E2A002A44134517C5104510661438
:1003F00067170130671FE400DE226716E716080062
:1004000044174517C5144510661466156717043060
:10041000671FE400DE226716E71608000310720C5F
:1004200070077202031C1C2A03191C2A0310720C89
:10043000013E7007F000212A0310720C013E700289
:10044000F00044134517C514451066146615671768
:100450000430671FE400DE2208004908083C031945
:100460004E174908073C0319CE164908063C0319E4
:100470004E164908053C0319CE154908043C0319DA
:100480004E154908033C0319CE144908023C0319D0
:100490004E144908013C03194D144908083C03193E
:1004A0004E171921D30D531A5314061706160516A5
:1004B0000514531C5E2A061354086D2AD31C632AA4
:1004C000061255086D2A531D682A051256086D2A12
:1004D000D31D0800051057086D2A87000800671F04
:1004E0000800E303031D080065186008E5186108AB
:1004F0006519620899000330E3000310E50DE51962
:10050000822A08000F30E3000130E500E6080319F5
:10051000932A0310E40D0318641464086605031994
:10052000822ADE220800671308008C1E0800E717E5
:100530004C141819CA146908E8006A08E9001A0876
:10054000EA006808583C031DB02A6908593C031D9D
:10055000B02A6A085A3C031DB02A0330EE00080096
:10056000EE0B08000330EE006808463C031DC02A6D
:100570006908671EC4006A08671EC6006712DD2A84
:100580006808453C031DC92A6908CA006A08CB00EF
:10059000DD2A68084C3C031DD42A6908E71EF000D8
:1005A000E7126A08F100DD2A6808413C031DDD2AD4
:1005B0006908F8006A08F900DD2A0800E001E10195
:1005C000E201641DEA2A6611C430E0007008E1000F
:1005D0007108E200E41CF32AE610C230E00047088C
:1005E000E1004808E200641CFC2A6610C130E0000B
:1005F0004408E1004508E2000800831203173B08A5
:100600008D003A088C00831603178C130C158B137E
:100610008B1B072B55308D00AA308D008C148B1747
:100620000C11831203130800431F08004313441FD7
:10063000C410F00A720A70020318F0004513C510C6
:10064000441FC5144510661466150430671FE40086
:100650006717DE226716E7160800C31F0800C313DA
:10066000441FC414F003720AF01BF0074513C510B1
:10067000441FC51445106614661567170430671FBC
:0A068000E400DE226716E71608000A
:100A00000A3050020318D00105308A0050088207CE
:100A10003F341834B634BC349934AD34AF34383440
:040A2000BF34BD34EE
:084000000D00000000000900A2
:02400E00CC03E1
:10420000000001000200AA00C80014003000FF00F6
:104210000000FF00FF00FF00410058001400FF00F5
:104220000000110012001300140015001600170002
:10423000060019001200FF00FF00FF00FF00FF0052
:10424000FF00FF00FF00FF00FF00FF00FF00FF0076
:10425000FF00FF00FF00FF00FF00FF00FF00FF0066
:10426000FF00FF00FF00FF00FF00FF00FF00FF0056
:10427000FF00FF00FF00FF00FF00FF00FF00FF0046
:10428000FF00FF00FF00FF00FF00FF00FF00FF0036
:10429000FF00FF00FF00FF00FF00FF00FF00FF0026
:1042A000FF00FF00FF00FF00FF00FF00FF00FF0016
:1042B000FF00FF00FF00FF00FF00FF00FF00FF0006
:1042C000FF00FF00FF00FF00FF00FF00FF00FF00F6
:1042D000FF00FF00FF00FF00FF00FF00FF00FF00E6
:1042E000FF00FF00FF00FF00FF00FF00FF00FF00D6
:1042F000FF00FF00FF00FF00FF00FF00FF00FF00C6
:00000001FF
